:020000040800F2
:10500000381A0020D5500008ED820008FD7A00080B
:105010000000000000000000000000000000000090
:10502000000000000000000000000000A18F000848
:10503000000000000000000095880008B9900008FA
:10504000E7500008E7500008E7500008E750000864
:10505000E7500008295B0008E7500008E750000807
:1050600000000000E7500008515A0008E75000080F
:10507000E7500008697F000800000000E7500008C2
:1050800000000000E75000080000000000000000E1
:10509000E750000800000000E7500008E750000853
:1050A000E7500008E7500008E7500008559800084E
:1050B000E7500008E7500008000000000000000072
:1050C0000348854600F060FC0048004745A50008FD
:1050D000381A00200448804704480047FEE7FEE7EE
:1050E000FEE7FEE7FEE7FEE755910008C150000825
:1050F00030B50B46014600202022012409E00D4670
:10510000D5409D4205D31D469540491B25469540F7
:1051100040191546521E002DF1DC30BDF0B51FB40C
:105120000646002082B005464024019100901BE015
:10513000019922460F46304600F04EFB049A059B2B
:10514000801A994110D310461946224600F034FBCC
:10515000361A8F410197224601200021009F00F05E
:105160002BFB38184D4100902046641E0028DFDCE0
:10517000019B00982946324607B0F0BD03460B4319
:105180009B0703D009E008C9121F08C0042AFAD2FD
:1051900003E00B780370401C491C521EF9D2704783
:1051A000D2B201E00270401C491EFBD270470022BF
:1051B000F6E710B513460A4604461946FFF7F0FF16
:1051C000204610BD30B504460020034600E05B1CBD
:1051D000934203D2E05CCD5C401BF8D030BDF8B503
:1051E00002464A40D40F42004B0052085B089A42E4
:1051F00002D20246084611464A0023D0C30D4A0097
:10520000DDB2120EAD1A202D35DA49020126490A07
:10521000F6058A19002C00D0524220214F1B11465E
:10522000B9402A411018C20D9A4221D0002C17D043
:10523000012D08DCDA05801AD20F8019D207DBB203
:1052400000F0F6FAF8BDDA05801A012340001B06CB
:10525000C01880185A428018CA0F1043490007E04E
:105260004908C2071143DA05801A801940088018DE
:1052700000F0D6FAF8BD61000122511A001BF7E7D1
:105280000122D2075140AAE70122D2075040A6E7E7
:1052900070B502464A40D50F40004A00ED0740086D
:1052A0005208002814D0002A12D0C40DD30D410298
:1052B0000120C0055202490A520AE41A09181218BC
:1052C0007D34914201D3641C00E04900002C01DAD6
:1052D000002070BD0023914201D3891A0343400886
:1052E00049000028F7D100290AD0914202D10121BA
:1052F000C90705E0914201D2012101E00121C94322
:10530000E005C018401900F08BFA70BDF0B50746F3
:105310000846584087B0C00F049048000E46590018
:1053200040084908BC1A884105D2384631461E4615
:1053300017460B4602465800400810434CD0300D2B
:10534000039040055900400D490D0590401A029008
:10535000402872DA18030121000B09050843019067
:1053600004980092002805D00199524200208841FB
:1053700000920190029840210A1A0199009800F0C9
:105380001BFA05460C466B4607CB00F036FAC019EF
:105390007141039A0E0D0023D71756401A467A40E2
:1053A000164344D0049A002A2DD0029A012A039A67
:1053B00015DC1205C01A914101263605001C714109
:1053C000D20F059ED2070093019202962A462346E9
:1053D00000F074FA07B0F0BD38463146FAE716051A
:1053E000224A0F46B218C01AB74101210905001C14
:1053F0004F4100187F41114618187941E20F1043C0
:105400006D19644113E0E2076D0815436408C20793
:105410001443039A01261205C01A91413605001C57
:105420007141CE07400830434908C01851412A460F
:10543000234600F036FACDE7FFE70498012240004A
:10544000C117121A00238B4104983146C417381A29
:10545000A141EEE730B40124E407634030BC55E7D6
:1054600030B40124E407614030BC4FE70000E0FFA6
:10547000F0B51FB488B00B990998002448400999E9
:10548000C00F490049080991C0070B9900904900D5
:1054900049080B9109990898A64608431CD00B9916
:1054A0000A98084318D0099801244000420D48008A
:1054B000410D099824050003000B204309900B9827
:1054C0000003000B20430B9050181C494018002289
:1054D00001901446104605E0002001460DB0F0BDD5
:1054E000032801DA034600E003239C46C11A0AAEF2
:1054F0000AE05F0008ADED5B4F00F75B7D430027DE
:10550000AA187C41491C5B1E6145F2DD410004ABD9
:105510005A522104120C0A43240C401C0828DFDBD9
:10552000019802900099704601910090059B049AA1
:105530000799069800F0C2F9D0E700000DFCFFFFC4
:10554000F0B50C465C4085B0E40FE40703944C00D2
:1055500000266408590094464908024602962243F0
:1055600021D062460A431ED06200570D4A000E0346
:105570002303550D012402462C492405781B1B0BDF
:10558000360B401823432643614600901C46501AB0
:10559000B44103D30098401C009002E09218009898
:1055A0005B41002803DA0020014605B0F0BD002071
:1055B000012109050746864611E064461D46141B75
:1055C000B54106D36546521BB341744607430C43AD
:1055D000A646CD0740084908284392185B41054676
:1055E0000D43EAD11046184313D060461946504087
:1055F0007140084306D06046101AB34106D201221A
:10560000002306E000220123DB0702E00122D2434F
:105610005310009874460105381C6141029C039D9B
:105620000019694100F03DF9BFE70000FD030000EB
:10563000C217C10F504010B54018CA079623002169
:1056400000F0F6F810BD10B500229623114600F0C8
:10565000EFF810BD0EB5C217C10F5040CA07401871
:105660000021054B0293019200910A460B4600F07F
:1056700025F903B000BD0000330400000EB5054954
:105680000291002100910A460B46019100F016F9A3
:1056900003B000BD33040000410040020122400A73
:1056A000D205090E80187F2901DA0020704796295B
:1056B00003DC9622511AC8407047963988407047DB
:1056C00070B5CD0F4A0009030123090B1B051943CF
:1056D0000B4BED070024520D9A4201DA002070BDF9
:1056E000074B34339A4203DC9A1A00F075F802E053
:1056F0000449511888402C43F1D0404270BD00004D
:10570000FF030000CDFBFFFF4A0009030123090B43
:105710001B051943094B10B5520D9A4201DA0020BE
:1057200010BD064B34339A4203DC9A1A00F054F849
:1057300010BD03495118884010BD0000FF03000050
:10574000CDFBFFFFC20FD207400040080BD0C10DB8
:105750000723DB01C91840020905400A1143C208AA
:10576000400711437047002001467047CB0FDB070D
:10577000490010B5490802460A4307D00A0D07241C
:105780000903E401090B121B002A01DC002010BDF3
:10579000C900440F0C43C100E018D205801800F086
:1057A0003FF810BD0122D207002800DB101A0029A3
:1057B00000DB511A8142704710B5202A04DB0146F4
:1057C000203A9140002010BD914020239C1A0346AE
:1057D000E3401943904010BD10B5202A04DB084671
:1057E000203AD040002110BD0B46D340D0402024A9
:1057F000A21A91400843194610BD10B5202A06DBB5
:10580000CB170846203A1041C1170B4306E00B4660
:105810001341D0402024A21A91400843194610BDDC
:10582000002904DA401C490001D1400840007047BB
:1058300070B40024050C05D11024000402D1002905
:1058400021D01124050E01D100020834050F01D129
:105850000001241D850F01D18000A41C002801DB5C
:105860004000641C002908D020252E1B0D46F54061
:10587000A14000D001212943084301061B1B000A57
:10588000DB1D02D5002070BC7047DB05181880189E
:105890000029F8DA401C4900F5D170BC40084000EE
:1058A000704710B5002B08DA0024401C61419218A3
:1058B0005B411A4301D14008400010BDF0B51FB450
:1058C00082B005460C0003D0084604F07DF802E0E3
:1058D00004F07AF820300246009021462846FFF76F
:1058E0006BFF049B059A04460F4618431143084377
:1058F00014D0184610431BD0009840210A1A1846AD
:105900000599FFF769FF05460E46009A0599049828
:10591000FFF752FF084305D0012004E02046394636
:1059200007B0F0BD0020C11705430E432C43374399
:1059300000990E986305401A7905E40A00220C4389
:10594000FD0A0A3002D500200146E9E701051019D9
:1059500069410C9C0D9D00196941FFF7A2FFDFE72B
:1059600010B5002904DB0124E40740428C412146A4
:10597000002B04DB1C460123DB075242A341994262
:1059800000D1904210BD0000064C0125064E05E0F6
:10599000E36807CC2B430C3C98471034B442F7D350
:1059A000FFF792FBC0A80008E0A8000838B504463D
:1059B000064805490068FFF79BFB604300E0401E76
:1059C00000900028FBD138BD40420F001C01002090
:1059D000F8B50446006881688907890F012902D15A
:1059E0000168C90722D18168114A1026114001259A
:1059F00000290ED18168294381600120FFF7D6FF7D
:105A000000F082FF07460CE000F07EFFC01B0A2872
:105A100007D9606D30436065A06D2843A065012003
:105A2000F8BD20680068C043C007EDD10020F8BD74
:105A30001700008010B500231A4603E0845CE318C9
:105A40009BB2521C8A42F9D3D84380B210BD0000E9
:105A500010B5034800F018FD024800F015FD10BD18
:105A6000D81500209015002030B5446C1C252C4022
:105A70000125A540046C6560046863608368102B91
:105A8000036803D099600068C26030BD9A60006806
:105A9000C16030BD1449012048720A4602205E32BE
:105AA000507203203C3A507204200E3A50720F4854
:105AB0000D4B0078087022310870203108770C49AE
:105AC0005A1C0878587149789971233318715971A3
:105AD000203318775977107551751A461E32107594
:105AE000517510765176704750110020D700002074
:105AF000F400002010B503F02BFA202003F0D2FAB6
:105B0000012004F079FA002003F0CCFA044804F0F4
:105B100017F9044804F0C6FB002004F0FBFB10BD9D
:105B2000C000002083800000F8B505200121000797
:105B300000F0DAFE0025184C002800D06560174EF2
:105B40000221304600F0D0FE00281DD10120207037
:105B50001348808F00280ED00127BF02002239464B
:105B6000304600F0CAFE0A2004F09CF801223946B3
:105B7000304600F0C2FE0B48656000880A214843A9
:105B80000949088003F078FE012000F0E5FD0220BD
:105B900000F0E2FDF8BD00001001002000040050FC
:105BA000500D0020E4000020F000002070470000AD
:105BB00010B5084900224A6107494B684C15234338
:105BC0004B604B68082423434B60C009C00102604E
:105BD00010BD000020160020002002407FB50025E7
:105BE0000C460646039500F087FDE009029003A9E4
:105BF00001960095684600F017FD002804D000F0DB
:105C00004FFD002004B070BD00F04AFD0120F9E70F
:105C100010B5002302E0C45CCC545B1C9342FAD361
:105C200010BD000010B5214A00219069C30520482D
:105C300004D54169022319434161911593699B057C
:105C400005D54369012423434361630219439369E2
:105C50005B0505D54369082423434361E3011943E8
:105C600093691B0505D543690424234343616302FB
:105C7000194393699B0405D5436910242343436169
:105C80006302194393699B0304D5446920231C4391
:105C9000446119439369DB0305D5436940242343D9
:105CA0004361A0020143916110BD00000020024049
:105CB0002016002070B5054600F026FE0646184C5A
:105CC0000AE0681C08D0002D04D000F01DFE801BE7
:105CD000A84201D9032070BDA069C007F1D1A06915
:105CE000800701D50220A061A069C00511D4A06978
:105CF00080050ED4A06940050BD4A069000508D426
:105D0000A069800405D4A069800302D4A069C003FF
:105D100003D5FFF787FF012070BD002070BD000094
:105D200000200240F8B51746002605460C4600F054
:105D3000E3FC09E029460220226800F0BFFC0028AD
:105D400004D1241D2D1D361DBE42F3D300F0A8FC46
:105D5000BE4201D20020F8BD0120F8BD10B50849AF
:105D600002460020054B497905E044001C5B944243
:105D700003D0401CC0B28842F7D310BD7812002077
:105D80005800002010B500F0B4FD10BD10B5094852
:105D900000F0C6FF80B2FFF771FC074A074BFFF720
:105DA00067FB0022064BFFF7CBFBFFF7ADFC80B291
:105DB00010BD000088140020F853E3A59B843E40EA
:105DC00000408F4070B5364934488A7F0275C97FDC
:105DD000417534490A780276497841762F49052081
:105DE000133148720A2004F04DFA7D20C00004F0FF
:105DF00063FA2A49002213310C2004F02DFB002104
:105E00000C2004F03BFB022004F08CFA264D244CBD
:105E100000210F2004F0B6F928422063F8D0206B4F
:105E2000411C38D0400435D58122D20100210F20F9
:105E300004F0E7FA0021102004F0A4F94106174805
:105E4000490E0022633004F0D3F9144D6335687AAB
:105E500005281FD102221349681DFFF7B3F9002856
:105E600018D10F48AE7C66710422691C4430FFF7DC
:105E700085F929461331084672000D465130FFF767
:105E80007DF96079294642000448DF30FFF776F952
:105E90000320207070BD02F04DFA0000B111002007
:105EA00058000020F400002000D0272410B5084836
:105EB00000F096FA0A21064800F032FA044800F091
:105EC0001DF9800503D5024800F01AF980B210BD13
:105ED0002C140020F8B52F4D00220121284600F097
:105EE0000CFDFFF7E3FFFFF7AEFB2B4E3146FFF74C
:105EF000CFF92A4C0122A0601146284600F0FDFC93
:105F00002749A068002588423EDB2078254F0028DD
:105F100015D02570FFF7CAFFFFF795FB3146FFF755
:105F2000B7F9A060FFF70EFC00223B46FFF792FA9C
:105F300000221D4BFFF79CFAFFF718FC6060A06879
:105F4000FFF700FC00223B46FFF784FA174A184B84
:105F5000FFF78EFA06460F466068FFF7F3FB134A19
:105F6000144B5242FFF784FA32463B46FFF7CEF914
:105F7000FFF7FCFB10496060884201DD616004E0CE
:105F8000FF21C905C84200D365606068FFF784FB44
:105F9000C0B2F8BD0004005000401B443000002097
:105FA0000000604000000C4000E0644033333333B5
:105FB00033B33040CCCCEC3F0000C842F8B50546C6
:105FC00004464035287C0026012808D0012028748A
:105FD000206881688907890F01290ED101E002201C
:105FE000F8BD0168C90708D0606D202108436065CD
:105FF0000126002028743046F8BD616DFF22013271
:106000009143022211436165C1688907890F00919C
:10601000C16889088900C1602068816892071143BE
:10602000816000F071FC07460EE000F06DFCC01BC3
:106030000A2809D9606D0221884310210843606550
:10604000002028740120F8BD206880680028ECDB5F
:106050002068C168009A1143C160606D80088000AB
:10606000401C6065C5E70000F8B506460D464036A1
:10607000317C01290DD00121317401688A685207F1
:1060800009D5416D20221143416500203074012063
:10609000F8BD0220F8BD174B6A68D80547109A4230
:1060A000154C8A6A2B6812D05B035B0B1A438A6219
:1060B0002968490305D5A1680143A1600A20FFF7BB
:1060C00075FC2868800312D5A06838430EE05B0396
:1060D0005B0B9A438A622968490302D5A168814310
:1060E000A1602868800302D5A068B843A0600020A2
:1060F0003074F8BD0110000000270140406D70476A
:106100000068006C7047000070B5040006D0606D38
:10611000264600254036002802D006E0012070BD4A
:10612000A5653574204600F0D3F8606DC00603D431
:1061300021688868400705D5606D102108436065B7
:106140003574EBE7606DFF22013290430222104369
:10615000606588688207920F5B48012A02D10A684D
:10616000D2072BD1032362689B079A4205D05B427A
:106170009A4202D05B009A4209D10A6992009208C1
:106180000A6121680A6963681A430A610CE00A69B6
:10619000920092080A6181680F2292049143816003
:1061A00081686268114381602168CA6818239A4334
:1061B000CA602168CA68A3681A43CA60816801225C
:1061C0005206914381608168A28E5206114381601C
:1061D00020688168C90004D4816801221207114334
:1061E00081602068C168394A1140C1602069E16856
:1061F000022825D000200143204620300278037B6E
:1062000052035B001A431143226B1143A2699203AC
:106210001143E269D20311432268D3681943D16064
:10622000616A0A46FF3AC23A05D0A26A114322685F
:10623000D3681943D16042780121012A02D00BE0D2
:106240000420D8E70078002823D0606D2022104376
:106250006065A06D0843A065E06B012820681FD031
:106260000169C90703D00169490849000161206833
:106270004169C908C900416120684169A26B1143A5
:106280004161A565606D80088000401C606500204C
:1062900070BD2068C26801231B041A43C260DBE79B
:1062A0000269FF239B009A43026120680269236C04
:1062B000A66C1A43636C33431A4302612068026977
:1062C0000A430261D3E70000002701401902FEFFE4
:1062D00010B586B0044614216846FEF768FF0E49E3
:1062E0002068884216D10D48416B42151143416325
:1062F000C16A01221143C162C06A6946104005901B
:106300000220009003200190002002900520000749
:1063100000F02EFA06B010BD00240140001002402B
:10632000F8B504464069254640350E4608280BD08E
:106330002068C068C00709D0606D202108436065EF
:10634000002028740120F8BD082700E00C2700F089
:10635000DBFA009011E0701C0FD0002E05D000F089
:10636000D3FA0099401AB04207D9606D042108435E
:106370006065002028740320F8BD2068006838425A
:10638000E9D0606D01214902084360652068C16859
:1063900009058A0F0C21002A1BD12022125D002A38
:1063A00017D10268120714D5826853070122002B07
:1063B00008DB43688B434360606D130298431043CE
:1063C000606506E0606D202318436065A06D104392
:1063D000A065A069002801D1206801600020F8BDF7
:1063E00070B50446216800208968490721D42546F4
:1063F0004035297C01291CD001212974E16901293A
:1064000004D02046FFF7E4FA002811D1616D0A4A52
:106410001140FF220132114361650021A1652974F9
:1064200022681C21116021688A6804231A438A604B
:1064300070BD022070BD0000FEF1FFFF70B50024AA
:10644000014620314A79022A03D00421C163012484
:1064500018E0026813680E25AB43136002681368E6
:106460005B085B001360436C1C221340012215463D
:106470009D40036C5D604A7100220A71816B0029A6
:1064800000D08847204670BDF0B4016C0D680168EB
:106490000C68466C1C2304221E401746B7402F424E
:1064A0000ED067070CD50C68A40602D40C68944380
:1064B0000C60416C19408A40016C4A60016B1AE023
:1064C0000227B74002462F402032002F17D0A707DF
:1064D00015D50C68A40605D40C680A25AC430C60DD
:1064E00001215171446C02211C40036CA140596090
:1064F00000211171C16A002918D0F0BC0847082793
:10650000B7402F4212D0240710D50C680E25AC439B
:106510000C60446C01211C400B46A340046C63607A
:10652000C163517100211171416BE4E7F0BC704708
:1065300070B504003CD01F48256814212818FEF7C8
:10654000D7FD800060641C48206402212046203072
:106550000246417129681948E3680140A0686669EC
:106560001843236933431843A3691843E369184365
:10657000236A1843084328600121A06889038842E0
:1065800010D00D488030836A656C1C210D400F26A9
:10659000AE40B3438362656C63680D40816AAB4073
:1065A0000B4383620020E06301215171107170BDC3
:1065B000012070BDF8FFFDBF000002400F80FFFF0B
:1065C000F8B504468C46203001790025012909D010
:1065D0000126067141790027012905D0077102259E
:1065E0002846F8BD0220F8BD02214171E76320680A
:1065F000016849084900016061462046FFF734FA06
:10660000206B00282068016801D00E2205E00422DA
:1066100091430160206801680A22114301602068EB
:10662000016831430160DBE7F8B51A4E0546307C5E
:106630000F46012807D0012030741748FFF73AFBB6
:10664000010002D021E00220F8BD0020C0433860E4
:106650006C6814E02046FFF7ABFA0F48FFF72AFBFF
:1066600001460E48426808239A4342604268431537
:106670009A434260002901D03C6006E08034A8685B
:106680006A68C0018018A042E4D80020307408462F
:10669000F8BD00002016002050C30000002002407A
:1066A00005484168022211434160416801221143BB
:1066B000416000207047000000200240F8B50C4CFB
:1066C0001646207C0F46012808D001202074094876
:1066D000FFF7F0FA0025002802D006E00220F8BDFE
:1066E00065613E600348FFF7E5FA2574F8BD0000D8
:1066F0002016002050C3000011484168C9070BD084
:10670000EFF3108172B60F4AC2600F4AC26081F384
:1067100010884168C9070ED1416889070DD5EFF38C
:10672000108172B6094A0261094A026181F3108838
:106730004068800701D501207047002070470000A5
:1067400000200240EFCDAB8905040302BFAE9D8C53
:10675000161514137047000010B504494A69024227
:1067600002D04861FFF7F6FF10BD000000040140B1
:10677000F8B500230124A2E027469F403A4070D09C
:106780004D68022D01D0122D14D1DD08AD002D1859
:1067900000952D6A5E07AC46F50E0F26AE46AE405C
:1067A0006546B543AC460E697546AE4065462E4318
:1067B000009D2E624D68012D05D0022D03D0112DB4
:1067C00001D0122D16D185680326AC465D00AE4679
:1067D000AE406546B543AC46CE687546AE406546AC
:1067E0002E43866046680D79BE43ED06ED0F9D4051
:1067F0003543456006685F000325BD40AE46AE43A5
:106800000D79B446AE07B60FBE4065462E4306600E
:10681000C6687546AE438D68BD403543C5604D685A
:10682000ED004BD5294D6E6B26436E639E08284DB7
:10683000B6007519AC46AD689E07360F0F27B740F6
:10684000BD4305273F07B84201D1002715E0214F7E
:10685000B84201D1012710E01F4FB84202D10227F0
:106860000BE02BE01D4FB84201D1032705E01C4F80
:10687000B84201D1052700E00627B7402F436546FF
:10688000AF60184D2E684F689643FF0300D516433E
:106890002E606E684F689643BF0300D516436E6046
:1068A000AE684F689643FF0200D51643AE60EE68AF
:1068B0004F689643BF0200D51643EE605B1C0A6822
:1068C0001546DD4000D057E7F8BD0000001002403B
:1068D000000001400004005000080050000C00506F
:1068E000001C0050000401400069084000D0012055
:1068F000704742694A4042617047002A01D0816175
:1069000070478162704700000148006870470000CE
:106910001801002002480168491C0160704700000E
:106920001801002010B508480024016840221143D6
:106930000160204600F00AF8002801D0012401E09F
:1069400000F01AFA204610BD0020024070B505463E
:1069500009487D210024C9000068FEF7C9FB00F04A
:10696000AFFE002801D0012404E000222946501E79
:1069700000F022FA204670BD1C01002070477047CD
:10698000F8B55D4CA078401CA07001202071E08A11
:10699000401CE0825948008802F040FB584DE888CE
:1069A000FEF751FE5749FEF773FC574E0746316814
:1069B000FEF715FC30600120616AC005814203DBEF
:1069C0003846FEF761FC6062607800280CD1022135
:1069D0004E48FFF789FF02004D494E4814D000226F
:1069E000FFF78BFF0020606302214848FFF77CFF20
:1069F000002850D000206063434E4749376847481D
:106A00008F4259DD012158E00122D1034148FFF7AF
:106A100074FFE888FEF717FE3A49FEF739FC616B10
:106A2000FEF7DDFB3E4960638842DDDD3448012727
:106A3000F926403000900A213046FEF759FB002924
:106A400003D133493348FFF79DF902212F48FFF75F
:106A50004BFF002801D0002701E0002F12D10221B6
:106A60002A48FFF741FF00280CD103F03DFE0099B2
:106A70000120888003F094FE642003F013F92A4972
:106A80002848C8600A2003F00DF93046761EF6B299
:106A90000028D0D1A8E7E888FEF7D5FD1949FEF710
:106AA000F7FB616BFEF79BFB204960638842A3DB29
:106AB0001D481C49C1609FE700210170688F401E7E
:106AC000FEF7B6FD3946FEF76DFE04D86079002862
:106AD00001D0012000E0002015490870688FFEF702
:106AE000B2FD3168FEF75EFE04D26079002801D065
:106AF00003F0BEFDF8BD0000D400002074000020AB
:106B0000500D002000007A441401002000040050C1
:106B100000800000000000500000F0425E000020F5
:106B2000000040400400FA0500ED00E00000A04035
:106B30006C000020704770B505000DD002202C4677
:106B40002034A073284601F017FA284600F0BEF85A
:106B50000020A073607370BD012070BD7047704746
:106B600010B5044600680168C943C90708D18168A7
:106B7000C943C90704D1012141602046FFF700FF46
:106B800020680168C943890708D48168C943890717
:106B900004D4022141602046FFF7F0FE206801681E
:106BA000C943490708D48168C943490704D404216B
:106BB0004160204600F0DEF820680168C9430907FB
:106BC00008D48168C943090704D4082141602046DC
:106BD000FFF7B0FF20680168C943C90608D481687F
:106BE000C943C90604D4102141602046FFF7C7FEFF
:106BF00020680168C943890608D48168C9438906A9
:106C000004D4202141602046FFF7A9FF20680168D5
:106C1000C943490608D48168C943490604D44021C0
:106C200041602046FFF79AFF10BD0000F8B5040050
:106C300005D025462035A87B002802D006E001209B
:106C4000F8BD00206873204600F052F80220A873B7
:106C50002068C26884466368012B04D00120A16AC1
:106C6000C005814201D11E208243154861698142DD
:106C700001D0144802401448A66802401846304328
:106C8000676A266A3E433043A66A30431043012BAD
:106C900003D00122D205964203D12369E2681A4348
:106CA0001043074A914205D0A2691143E2690243A9
:106CB000084610436146C8600120A8730020F8BD53
:106CC000FFFF00003F1FFFFFF8F119FF10B500683C
:106CD0000549884207D10548816B4900490881630D
:106CE0000D2000F055F810BD007C0040001002405F
:106CF00010B50068084988420CD10848816BC2046D
:106D000011438163002201210D2000F055F80D2070
:106D100000F048F810BD0000007C00400010024068
:106D20000068C0697047000070B502240346203334
:106D30009C730F4C2568E604354325600468E568BC
:106D4000B6123543E5600568AE6801242643AE609F
:106D500005682E6926432E610568A96101684A61AC
:106D6000006801690422114301619C73002070BD19
:106D700000040140704700000448416B01221143A8
:106D80004163816B0204114381637047001002402C
:106D9000C106C90E01208840014908607047000003
:106DA00080E100E0C106C90E012088400149086069
:106DB0007047000000E100E010B501F099FA10BD45
:106DC00002494A6882434A607047000000700040F0
:106DD000024801688215114301607047007000404D
:106DE00002494A6802434A60704700000070004050
:106DF0000548016802221143016004480169042228
:106E00001143016130BF70470070004000ED00E0A9
:106E10000A4B1A689208920002431A6008480369F4
:106E2000042213430361012906D040BF20BF20BFC5
:106E3000016991430161704730BFF9E7007000407C
:106E400000ED00E0F8B504460078544D800672D598
:106E5000524E0027403EB06BC00004D4B06BA90571
:106E60000843B06301274E480168C90511D4016881
:106E7000821511430160FFF747FD009005E0FFF721
:106E800043FD0099401A642837D845480068C0057A
:106E9000F5D532680321090560680A400140914236
:106EA00008D08103890F032904D13168890301D5F2
:106EB0000120F8BD2A69032109040A4022D00840B4
:106EC00090421FD0207880061CD528692A69884303
:106ED0000121C9040A432A612A698A432A61286177
:106EE000C0050FD5FFF710FD009008E0FFF70CFD7F
:106EF0000099411A2B48814201D90320F8BD286925
:106F00008005F3D561688803800F032805D13268B6
:106F10000005824301400A43326028690322616808
:106F20001204114008432861002F04D0B16B0120E6
:106F300000078143B1632078C00705D0E868A168E5
:106F4000800880000843E8602078800705D5E8685D
:106F50000C218843E1680843E8602078400706D5A3
:106F6000E86803218902884321690843E8602078A2
:106F7000000706D5E86803210903884361690843CF
:106F8000E8602078000606D5E86803218904884374
:106F9000A1690843E8600020F8BD000040100240ED
:106FA0000070004088130000F8B50E4605007DD043
:106FB00053480068C007C00FB0420AD25048016869
:106FC00049084900314301600068C007C00FB04262
:106FD00071D128784B4C800705D5E068F0218843B3
:106FE000A9680843E0602878C00752D06868022882
:106FF00017D0032818D02168012818D08905002946
:1070000059DAE168890889000143E160FFF77CFCF7
:1070100069680746022912D003291CD0012926D00D
:1070200033E021688903EAE721688901E7E7490736
:10703000E5E7FFF769FCC11B3348814223D8E068CC
:107040000007800F0228F4D123E0FFF75DFCC11B8D
:107050002D48814217D8E0680007800F0328F4D13B
:1070600017E0FFF751FCC11B274881420BD8E068AD
:107070000007800F0128F4D10BE0FFF745FCC11B8E
:107080002148814201D90320F8BDE0680007800F44
:10709000F3D11B480168C907C90FB1420DD9016876
:1070A0004908490031430160006800E003E0C0077F
:1070B000C00FB04201D00120F8BD2878400706D5A6
:1070C000E068072109028843E9680843E0602878FE
:1070D000000707D5E0680721C90288432969C9006C
:1070E0000843E06000F036F8E168084A0906090F35
:1070F000515CC840064908600020FFF727FCF8BD36
:107100000020024000100240881300009EA80008E2
:107110001C010020044805490068C968044A490563
:10712000490F515CC84070471C010020001002400C
:10713000B7A80008044805490068C968044A8904DA
:10714000490F515CC84070471C01002000100240EC
:10715000B7A8000810B5184AD1680C2008400428C8
:107160000BD0082810D00C2810D050680004410F14
:107170000120C003491C884010BD1068C00601D51D
:107180000E4810BD0E4810BD0E4810BD88020E4BB3
:10719000000F185C0902D368890F491CDB0301D575
:1071A000084A05E01268D20601D5044A00E0044A04
:1071B0005043FDF79DFF10BD0010024000093D0047
:1071C0000024F40000127A00AEA80008FEB5050005
:1071D0007ED0FE4CE7680C20E668074001200004E2
:1071E00006402878C00747D0082F05D00C2F0AD1B9
:1071F00001200004864206D1206880033CD56868DF
:107200000028E5D038E0012069680004814203D1FC
:1072100021680143216011E0052301221B0492042F
:107220009942216802D111432160F1E78143216035
:107230002168014000912068904320606868002820
:107240000DD0FFF761FB009005E0FFF75DFB0099B3
:10725000401A64287AD820688003F6D50CE0FFF73E
:1072600053FB009005E0FFF74FFB0099401A64289C
:10727000F0D820688003F6D42878800755D50923F4
:10728000E868042F0DD00C2F01D1002E09D0002862
:107290003BD02168994301432160FFF735FB064647
:1072A00027E02168490701D5002891D061681F2295
:1072B000120291432A6912021143616021689943C5
:1072C00001432160FFF746FFE16809060A0F00E06D
:1072D00079E1BF49895CC840BE4908600020FFF7DA
:1072E00035FB002872D120E0FFF70EFB801B02283F
:1072F000B0D820684007F7D560681F21090288438D
:1073000029690902084360600FE0206840084000D6
:107310002060FFF7F9FA064604E0FFF7F5FA801B54
:10732000022897D820684007F7D42878C0065FD590
:10733000002F0CD0A869002849D02068FF21013116
:1073400008432060FFF7E0FA06462DE0C0E0206821
:10735000800502D5A8690028A7D0606807214903E5
:107360008843296A084360606068297F0002000A38
:10737000090608436060286A410B0120C003491CCC
:107380008840E16809060A0F9149895CC840914923
:1073900008600020FFF7DAFA002817D128E0FFF78D
:1073A000B3FA801B0228A3D820688005F7D560684F
:1073B000072149038843296A084360606068297F80
:1073C0000002000A09060843606011E0E1E021685C
:1073D000FF20013081432160FFF796FA064604E062
:1073E000FFF792FA801B022872D820688005F7D434
:1073F0002878794E000724D568690028306910D0B4
:10740000012108433061FFF77FFA009005E0FFF7A4
:107410007BFA0099401A02285AD830698007F6D5BD
:107420000FE0400840003061FFF76EFA009005E081
:10743000FFF76AFA0099401A022849D83069800794
:10744000F6D42878400765D500200290A06BC000D4
:1074500006D4A06B012109070843A0630120029014
:107460005E480168C90511D40168821511430160A5
:10747000FFF74AFA009005E0FFF746FA0099401A34
:10748000642825D855480068C005F5D5FF20AA68AE
:107490000130824203D131690143316111E00121A0
:1074A0008902002A07D005231B029A4203D13269C0
:1074B0000A433261EFE732698243326130698843BF
:1074C0003061A86800280FD0FFF71EFA009007E08F
:1074D0005EE0FFF719FA0099411A4148814257D8F6
:1074E00030698005F5D50DE0FFF70EFA009006E053
:1074F000FFF70AFA0099411A3948814248D83069A1
:107500008005F5D40298002804D0A06B012109075A
:107510008843A063686A002864D00C2F3ED00126FF
:1075200036060228206805D0B0432060FFF7ECF94A
:1075300005462FE0B0432060FFF7E6F9074604E078
:10754000FFF7E2F9C01B022822D820688001F7D497
:10755000E96AA86AE2680843296BFD231B049A4381
:1075600011430843E060206830432060FFF7CCF906
:10757000054604E0FFF7C8F9401B022808D8206838
:107580008001F7D52EE0FFF7BFF9401B022801D993
:107590000320FEBD20688001F5D423E00128F8D047
:1075A000E06801210904AA6A014091420BD10F2130
:1075B0008904EA6A0140914205D103218905084006
:1075C000296B88420ED00120FEBD00000010024051
:1075D0009EA800081C0100204010024000700040DE
:1075E000881300000020EFE770B5040007D00026E4
:1075F00025464035A662687C002802D005E00120BF
:1076000070BD2E74204600F02FF8022068742068A8
:107610000168402291430160A168606822690843C3
:10762000E16811430843616901220843A1695202DC
:1076300011400843E1690843216A0843A16A0843ED
:1076400021680860A0690421000C0840616A0843B1
:10765000216848602068C16992009143C1616665F4
:1076600001206874002070BD10B586B00446142156
:107670006846FDF79CFD10492068884219D10F48E3
:10768000416B821411434163C16A01221143C162FB
:10769000C06A002110400590E02000900220019077
:1076A0000320039002910491052069460007FFF72B
:1076B0005FF806B010BD000000300140001002402D
:1076C000094910B5401E884201D9012010BD074C60
:1076D00060610321081F00F00BFE0020A06107205D
:1076E0002061002010BD0000FFFFFF0000E000E06F
:1076F00070477047F8B502680446D069116893680E
:1077000005072D0F5BD0DD07ED0FFF2621360E405C
:107710002E4367D0C60706D0CE0504D501261662D3
:10772000E26F3243E267870702220426002F06DA5F
:10773000DF0704D027683A62E76F3743E7674707F8
:1077400006D5DB0704D023681E62E36F1343E367AB
:10775000020709D520220A402A4305D023680822BF
:107760001A62E36F1343E367E26F002A2FD08006AB
:1077700006D5880604D5216E002901D02046884709
:10778000E06F21688968490601D4000724D52046A6
:1077900001F0D0FE20688168490619D58168402231
:1077A00091438160E06E002812D020498163E06E31
:1077B000FEF744FE00280AD0E06E816B06E08506E5
:1077C00010D58D060ED5216E1CE020468847F8BDE9
:1077D0002046FFF78EFFF8BD2046FFF78AFF002006
:1077E000E067F8BDC50208D55B0206D5012000059B
:1077F00010622046FFF77CFFF8BD030605D50B0697
:1078000003D5616E0029E0D1F8BD4006FCD54806DD
:10781000FAD51368204640218B431360202161670D
:107820000021616600F069F9F8BD0000919400083C
:1078300010B5040003D0606F002802D007E00120DB
:1078400010BD002170200155204600F027F82420AB
:10785000606720680168490849000160204601F01E
:10786000B3FE0128ECD0606A002802D0204601F067
:10787000F1FC206841680922D202914341602068EE
:1078800081682A22914381602068016801221143A6
:107890000160204601F044FD10BD0000F0B587B046
:1078A000064614216846FDF782FC2C493068884260
:1078B00051D12B48416B0122920311434163C16AAC
:1078C00001221143C162C06A0025104005900320C7
:1078D000400200900220032701A9A1C104200490C6
:1078E000052069460007FEF743FF1F4C1D48A560B1
:1078F000E56081C48027E560A76020202561606184
:107900000002A0611848083CFEF712FE002801D0D2
:10791000FEF74CF9F466A662144C1248214614385E
:1079200020600320606010200831A1C16561A5615D
:10793000E56120462562FEF7FBFD002801D0FEF739
:1079400035F9B466002201211B20A662FFF734FA44
:107950001B20FFF727FA07B0F0BD000000380140F8
:10796000001002403000024090150020D815002081
:10797000F8B50446806F20284DD100290BD0002A8D
:1079800009D00123A0681B03984206D12069002872
:1079900003D1C80701D00120F8BD25466035287CF9
:1079A000012838D001202874582061650253002630
:1079B000E6672220A067E06E002819D01749C1624F
:1079C000E16E17480863E16E16484863E06E13469F
:1079D0008663676D21683A462431E06EFEF7F0FD5C
:1079E000002805D01020E0672E7420206067D2E7C1
:1079F0002E7420680168FF22013211430160206863
:107A0000816801221143816020688168402211430E
:107A100081600020F8BD0220F8BD0000ED94000850
:107A20002B950008A594000870477047FFB50446E1
:107A3000406F83B017460D4620285CD1002D0AD038
:107A4000002F08D0A168C001814207D12069002819
:107A500004D1E80702D0012007B0F0BD2046603015
:107A60000290007C012846D0029801210174002078
:107A7000E06721206067FEF747FF26464036019009
:107A8000378277820120A1680003814202D12069F8
:107A9000002802D02F46002511E000270FE0002229
:107AA0008021204601F0A4FE002815D1002F15D01A
:107AB0002168387888627F1C708A401E7082708AC4
:107AC000019B002806980090E9D100224021204621
:107AD00001F08EFE002808D00320BDE72888216829
:107AE000C005C00D8862AD1CE6E7202060670299E2
:107AF00000200874B0E70220AEE770470149024851
:107B0000C160FDE70400FA0500ED00E010B50524B2
:107B10002407002204212046FEF7EFFE0022082160
:107B20002046FEF7EAFE0A2002F0C3F801220421F3
:107B30002046FEF7E2FE0A2002F0BBF800220421F4
:107B40002046FEF7DAFE10BD10B5052424070022FA
:107B500004212046FEF7D1FE012208212046FEF72F
:107B6000CCFE0A2002F0A5F8012204212046FEF7EF
:107B7000C4FE0A2002F09DF8002204212046FEF7F0
:107B8000BCFE10BDF8B5002405260746254636077D
:107B9000002204213046FEF7B0FE0A2002F089F8E8
:107BA000012204213046FEF7A8FE6006040E0821DB
:107BB0003046FEF799FE002801D0641CE4B205208F
:107BC00002F077F86D1CEDB2082DE1D3002F03D041
:107BD000FFF79CFF2046F8BDFFF7B6FFFAE770B548
:107BE000052605463607002204213046FEF785FEAD
:107BF0000024E80901D0012200E0002208213046DB
:107C0000FEF77BFE6806050E0A2002F052F80122FC
:107C100004213046FEF771FE0A2002F04AF80022E5
:107C200004213046FEF769FE0A2002F042F8641C87
:107C3000E4B2082CDDD370BD10B505242407012261
:107C400008212046FEF759FE012204212046FEF7B6
:107C500054FE002208212046FEF74FFE0A2002F0C3
:107C600028F8002204212046FEF747FE10BD10B57B
:107C700005242407002204212046FEF73EFE0022B0
:107C800008212046FEF739FE0A2002F012F80122F0
:107C900004212046FEF731FE012208212046FEF78E
:107CA0002CFE0A2002F005F810BD70B505252D0741
:107CB0000024012208212846FEF71FFE062001F0BD
:107CC000F8FF012204212846FEF717FE062001F0E6
:107CD000F0FF07E0641CE4B2FA2C03D9FFF7C7FFFA
:107CE000012070BD08212846FEF7FEFD0028F1D1D5
:107CF000002204212846FEF700FE002070BD00008F
:107D0000F8B501F03DFB01F077FB4C480068C06915
:107D1000FEF73CF84A4D4B49A882898F4A4E002411
:107D200000291ED06A6A730348499A4202DB022284
:107D30000A7000E00C700A7801218902002A0CD038
:107D4000012A04D0022A06D0032A0AD105E0FF2224
:107D5000F532904201D2002200E001223046FEF7C7
:107D6000CCFD0121C9023046FEF7BEFD0127FF030D
:107D7000002825D036480460E879002803D1012086
:107D8000E87101F079FD2878632806D900220821DE
:107D90003046FEF7B2FD012205E0012208213046FF
:107DA000FEF7ABFD0022052039460007FEF7A5FDD2
:107DB000244D284E4035A88C274F012803D01CE0C5
:107DC000EC710022EAE725486946088072B68021F6
:107DD0002348FDF703FF002804D00222694620480B
:107DE000FDF7A0FF62B61FA001F0E4FDAC8402F035
:107DF000D7FC642001F056FFFE60688C012808D192
:107E000010486C84048002F0CBFC642001F04AFF2F
:107E1000FE60288C012806D12C8402F0C1FC64206D
:107E200001F040FFFE600748124A0188914202D1EA
:107E3000C088002800D1FE60F8BD000010150020A9
:107E4000D4000020500D0020000400506A000020E3
:107E5000140100200400FA0500ED00E0AAAA0000C9
:107E6000384A0008BDF8C8EBC9FDBCB6C4A3CABDFA
:107E70000D0A0000AA55000008B53721202000F0A7
:107E80006EF80321212000F06AF84021222000F042
:107E900066F80821232000F062F8AA21302000F0C3
:107EA0005EF80A48008FC1B2322000F058F8022173
:107EB000332000F054F85F21202000F050F868468D
:107EC00000F006F80A2001F0F4FE08BD500D002075
:107ED00010B501460F2000F021F8002800D0012045
:107EE00010BD10B50446FFF7A7FE3220FFF777FE5E
:107EF000FFF7DBFEE0B2FFF772FEFFF7D6FEFFF7FB
:107F00009BFE3320FFF76BFEFFF7CFFE0020FFF74D
:107F100039FE0446FFF7ABFE204610BD10B50C46F7
:107F2000FFF7DFFF2070012010BD70B50D4604463D
:107F3000FFF782FE3220FFF752FEFFF7B6FEE0B2F7
:107F4000FFF74DFEFFF7B1FE2846FFF748FEFFF7AB
:107F5000ACFEFFF78CFE0A2001F0ABFE70BD10B541
:107F6000FFF7E3FF012010BD10B50248FEF7F8FD52
:107F700010BD000088140020FEB50446002572B62E
:107F80000068394A831804D13849CD68032189042F
:107F90000D4081680191C168009141698669002B9B
:107FA00008D132484038836AC7043B438362836AFE
:107FB000BB4383620846304348D02B482368C34202
:107FC00005D12A48C368032292049343C360002961
:107FD00017D02068026901231A43026120684161B9
:107FE000FEF792FC0746FEF78FFC2168C01B09686C
:107FF000090703D47D21C9008842F4D921680820EB
:108000004860002E17D020680169012211430161E8
:1080100020688661FEF778FC7D270646FF00FEF7A4
:1080200073FC2168801B0968C90601D4B842F6D9DF
:108030002168102048600C482168C14206D10B48D5
:10804000C1680322920491432943C16020680169F9
:1080500049084900016121680198886021680098F9
:10806000C86062B6FEBD00000084FFBF4010024041
:108070001CB5002116480091144A01910260C163A9
:10808000120542608160072282630122026102467A
:10809000C16020321170FF235170C233436281628C
:1080A000117301638161042241634261C161FEF782
:1080B0002BF8084800908013019069460448FDF7AA
:1080C000D3FF00210248FDF779FF1CBD00240140C9
:1080D0002C1400200200000408B50848016B01229E
:1080E00011430163006B01211040009000220A201F
:1080F000FEF762FE0A20FEF755FE08BD00100240A2
:10810000F0B587B014216846FDF751F84C48C26AB3
:1081100004210A43C262C26A0A400592C16A8027EA
:108120003943C162C16A39400591C16A01252943B9
:10813000C162C16A29400591C16A02263143C16208
:10814000C06A2A463040059005201C210007FEF732
:10815000D4FB01223B493C48FEF7CFFB00223B49C0
:108160003948FEF7CAFB91210520002209020007C9
:10817000FEF7C3FB364801900024052069460095B0
:1081800002940007FEF7F4FA0320019005206946E7
:10819000009602940007FEF7EBFA0C2000901120E5
:1081A0000190032003900520029469460007FEF722
:1081B000DFFA10200090052069460396019502948D
:1081C0000007FEF7D5FA1120019002946946009548
:1081D00003941D48FEF7CCFA1E48019069460096AC
:1081E00002951948FEF7C4FA1B48009002946946AC
:1081F000019503941448FEF7BBFAE8026A4651C29F
:1082000069461148FEF7B4FA91200002009005205B
:1082100002946946019503940007FEF7A9FA69469E
:108220000948009702950194FEF7A2FA0022012165
:108230000520FEF7C1FD0520FEF7B4FD07B0F0BD37
:108240000010024001060000000400500830000049
:1082500000001110000021100836000010B50F4C6E
:108260000D482060FF20053060600020A060E060C5
:1082700020616061E0610121206249026062A161C8
:10828000A0620720E0622046FFF7AEF9206801688F
:1082900040221143016010BD00300140B81400209D
:1082A00000B585B014216846FCF781FF0E480D49E2
:1082B0000160E1214902416000218160C1600161EA
:1082C00081610C22C1614261016230214162012160
:1082D000090381634900C163FFF7AAFA01F0C6FAF6
:1082E00005B000BD003801401015002070470000A7
:1082F0008307FF22DB0E9A408907090E9940002868
:108300000BDA0007000F0838830808489B0018188C
:10831000C36993430B43C3617047830804489B00C0
:108320001B181868904308431860704700ED00E080
:1083300000E400E0BFF34F8F04490348C860BFF377
:108340004F8F00BFFDE700000400FA0500ED00E0DC
:10835000F0B589B0FA4806900A2001F093FF7D201D
:10836000C00001F0A9FFF74C0025A570A07B0C28E8
:1083700001D30B20A073F448E570F44E00783071FF
:10838000F349A079097840000843217D890008431A
:10839000F071E06AF070401CE06260793146B074C0
:1083A0004200B4310846A138FCF7E8FE062070729E
:1083B000E848E4490078B072207F307330461338C3
:1083C0008A7F0275C97F417560790022400031467D
:1083D000153002F041F8607900214000153002F0BC
:1083E0004DF8022001F09EFFF5712574E572012021
:1083F00060732573D848FEF793FC60840646E570E9
:108400006079FDF73BF9D54AD54BFDF731F801F01E
:10841000E5FB012300229B07FCF778FFFDF774F9C9
:108420000006C10C881980B20121C903A0848842CA
:1084300001D3401AA084CB48A0632079401C20714E
:10844000C548FEF76DFC2084C0480C300646423615
:1084500040300390ABE1C048FEF762FC2084C24F7D
:108460000BE0BD48FEF75CFC80B22084A18C884202
:1084700003D3BE4A8918884206D300210F2001F099
:1084800081FE38422063ECD0206B411C21D0400497
:108490007DD58122D20100210F2001F0B2FF7D2085
:1084A000C00001F009FF002001F0BBFE00211020F8
:1084B00001F068FE4106A548490E274600225030CB
:1084C000A16401F095FEA1485030417A0729C1D13D
:1084D00001E0FFF72FFF0222A549401DFCF772FEC5
:1084E0000028B7D102F01BF87965386502F004F86E
:1084F000F965B865F8786946401CF87093484D30C6
:1085000002790A704079487008880090F98B884297
:108510007ED1984F308A388003988A49808A488370
:108520008D48FEF7FDFB208401F03EFDFF22A16D8A
:108530005204E06D0023891858410206080A1043CE
:10854000410849000090080E0902216660667F48D4
:10855000636D0A30226D01F0B7FF6079E36D810031
:108560007A48A26D0818163001F0AEFF7748636EA6
:108570001230226E01F0A8FF744808214172E07C9D
:10858000002816D0714802227949553000E001E1F7
:10859000FCF718FE00280CD101206C492074C8712A
:1085A000A06C66311638C2B208466274EA30FCF735
:1085B000E5FD60790022800064491C3001F04CFF29
:1085C0006079002180001C3001F058FF009801F014
:1085D00052FE012001F0A6FE607202216648FEF7FD
:1085E00083F900287ED00021594801705548B1898F
:1085F0008186F289C286606BA06354485030C37C88
:108600001807000F032800D0A0741809E07400E0D8
:1086100071E0257101204B4BE07219875A87207356
:10862000608B5649FF30C33080B2608388420BD9DB
:1086300049424018608338887D21401C80B2C900BF
:108640003880884200D33D803E887D20C000618B09
:1086500070434018E0630890494830210778494842
:10866000E77300884843FCF7EEFF029030460A218A
:108670004843FCF7E8FF0299FCF70AFE7F21C90591
:10868000FCF7ADFDFDF708F880B23D497F1E08807C
:10869000B84201D101202073E6841620205EFCF749
:1086A000D9FF06460191208CFCF7E8FF364A374B8C
:1086B000FCF7DEFE04900F460898FCF7CBFF3B4624
:1086C000049AFCF7C7FE3246019BFCF71FFEFCF73D
:1086D000F7FF2064A08B00F0A1FC607A002803D093
:1086E0006EE0FFE701217FE700210F2001F04AFD46
:1086F0000006F9D564E0FDF731FB254A032111544A
:108700001049B2898A86F289CA8621498000603977
:1087100042180399098B11801D4A796B303A115028
:108720000A49FB6D40181630BA6D01F0CDFE786B2A
:10873000069988423BD206900098079037E00000E7
:108740003F420F0058000020D4000020C411002038
:1087500010010020E400002088140020B81E85EBE2
:1087600051B8CE3FA086010000D02724983A0000DF
:10877000F40000200C01002000040050E70300007A
:10878000EA000020EE000020F853E3A59B843E4061
:10879000081300203A4600210F2001F032FE6079D4
:1087A000E178401C814202D0002001F03AFD208C8B
:1087B000A18C884200D24EE6304A89188842FAD805
:1087C00001F0F2FB2E4A00210F2001F01AFE207961
:1087D000002810D02B490A2209885143814200D237
:1087E0002570207C00282ED027490B7848788A787D
:1087F000022B16D027E0A26B0699323A204691420E
:108800000DD2C179491CCAB21E49C27109884900FA
:108810009142E6D20799C18302212170E1E7E57117
:10882000DFE710280AD0194BC91C1818FCF7A6FC62
:1088300001F0B6FF642001F035FA4AE6C878FCF78B
:1088400002FF13490860104D00209C3D2B46227802
:108850006179183307E04600AF5B9E5BB74200D0FA
:108860000222401CC0B28842F5D32270044A002183
:1088700080320F2001F0C5FD09B0F0BD983A00002C
:1088800000D02724E400002014130020500D002005
:10889000F800002070470000F0B58DB0B548019099
:1088A0000020C0430A9000260A2001F0EBFC7D2046
:1088B000C00001F001FD0020AF4C0546A070AF4F95
:1088C000AF480B90AE480022C23885730146142091
:1088D00001F0C2FD0021142001F0D0FD022001F0C2
:1088E00021FD00210F2001F04DFC38422063F8D01B
:1088F000206B411C18D040047ED58122D20100217A
:108900000F2001F07EFD0021102001F03BFC41060C
:108910009B48490E0022801C01F06AFC9848801C8C
:10892000417A022902D008E1FFF704FD94480222AF
:108930009449C01DFCF746FC0028F4D101F0EFFD7E
:108940006165206501F0D8FDE165A065002E23D1A9
:108950000B998D48098A018089488749801E808A41
:10896000488301268948FEF7DBF92084608B88491B
:10897000FF30C33080B2608388420DD9494240182D
:10898000814960830888824A401C80B20B3208808B
:10899000904201D3002008800B98694682890A80A2
:1089A000C089488076490422C91C0846A238FCF7D1
:1089B000E5FBFF22A16D5204E06D002389185841A8
:1089C0000006090A01430846029101F054FC02998D
:1089D00048084000010E0002616620666848636D29
:1089E0009638226D01F070FD6548E36D9238A26DF6
:1089F00001F06AFD624800E0A1E08E38636E226EED
:108A000001F062FD5E490022A0393C2001F024FD06
:108A100000213C2001F032FD012001F083FC607256
:108A2000A0780121401CA0700520C9030007FDF7B4
:108A3000A9F955487D220188D20008465043029189
:108A4000628B0A398018E0630C9052480078E0731A
:108A5000049008B22085002803DA7D21C90040185F
:108A600020854D48302100884843FCF7ECFD0590F7
:108A70002820205EFCF7DCFD0599FCF709FC7F212E
:108A8000C905FCF7ACFBFCF707FE424980B2088041
:108A90000499491E884201D1012020730298E08484
:108AA0001620205EFCF7D6FD05910690208CFCF781
:108AB000E5FD3A4A3A4BFCF7DBFC079104900C9831
:108AC000FCF7C8FD079B049AFCF7C4FC059B069ABB
:108AD000FCF71CFCFCF7F4FD2064A08B00F09EFA70
:108AE00000990198814210DA00290ED0244904220D
:108AF000C91C0AA8FCF742FB0220207029480A2161
:108B000000784843A07200980190607A002805D14F
:108B100000210F2001F036FB0006F9D5802200214C
:108B20000F2001F06EFC00206D1CEDB26070032D73
:108B300000D2C7E6002E08D017E00120F4E71A4A59
:108B400000210F2001F05DFCF7E7A18B17480029F9
:108B500002D00288914201D90188A18388B21449C8
:108B6000401E09884843134908800A98E0830DB0E5
:108B7000F0BD00003F420F005800002000D0272425
:108B800012120020F40000200C01002088140020A4
:108B9000E7030000EA000020EE000020F853E3A500
:108BA0009B843E40E400002000902724E000002049
:108BB000DE000020DC000020F8B5334931480860B1
:108BC00001F092FD32483149418001464031097936
:108BD000304C0906090E304F617003D0C18800295E
:108BE00008D009E0C7800121C1870A2141870021FF
:108BF000818701E06421C180018F0A2901D9022106
:108C00000187C18E3C2901D93C21C186234A89B202
:108C10001170C18F6171818FA171817AE170858836
:108C2000052125626181C6883046FCF761FAA08182
:108C300001462846FCF75CFA8800081885B21648F9
:108C400025816843FCF71AFD154A164BFCF778FCA2
:108C5000FCF75AFDE081658231463846FCF748FA58
:108C600020820146C820FCF743FA60830120E0829D
:108C7000FDF78CF8A082E2890B490C48FEF754F806
:108C8000F8BD0000A5980008500000201302000065
:108C9000500D0020D4000020E80300000000002058
:108CA000F853E3A59B843E40FF7F0000881400201A
:108CB000F0B5964D85B001202880954FC820954C81
:108CC0003880207A401C2072C00706D0A08B411E3D
:108CD000A183022801D2C820A083A08B00F09EF9B6
:108CE0000A2001F0CFFA7D20C00001F0E5FA022150
:108CF0008948FDF7F9FD002838D000208749800019
:108D00000978884E49000843854909780843B072BC
:108D1000102070728448C1887D20C000FCF7E8F9FB
:108D20007073824880490078B07330460B308A787F
:108D30000270C9784170411C7B482030027ECA70A5
:108D4000407E087178482230027E4A71407E8871E8
:108D500000220C39152001F07FFB0021152001F0C5
:108D60008DFB022001F0DEFA714E03E00120C5E721
:108D7000FEF7C6FF00210F2001F004FA3042206305
:108D8000F6D0206B411C7DD040047CD58122D201DD
:108D900000210F2001F035FB0021102001F0F2F935
:108DA00041066048490E00225030A16401F020FACB
:108DB0005C4E5036707A112865D102225D49701DD3
:108DC000FCF700FA00285ED1F01E027969460A70AD
:108DD00040794870B17A2980C820FCF789F9388039
:108DE000307BA083544DB01E008A28804949301F33
:108DF000808A48835148FDF793FF80B22084039016
:108E0000608B4F49FF30C33080B2608388420CD9F9
:108E100049424018608328884949401C80B20B3180
:108E20002880884201D3002028802D887D20C00022
:108E3000618B68434018E0630190424806782846F9
:108E40000A3800B2E6732085002803DA7D21C900C4
:108E500040182085388830214843FCF7F4FB07464A
:108E60002820205EFCF7E4FB3946FCF711FA7F214D
:108E7000C905FCF7B4F9FCF70FFC324980B2088051
:108E8000761E01E03FE03CE0B04201D101202073BA
:108E9000E5841620205EFCF7DDFB02900F46039868
:108EA000FCF7ECFB284A294BFCF7E2FA05460E4694
:108EB0000198FCF7CFFB2A463346FCF7CBFA3B463A
:108EC000029AFCF723FAFCF7FBFB20646846008853
:108ED000E083144813495030807C63316071420054
:108EE00008460D465130FCF749F9607929464200A1
:108EF0000C48CC30FCF742F9A08BFF2801D00320AE
:108F0000207005B0F0BDFFF715FA0000E400002066
:108F1000EE0000205800002000040050D90000207E
:108F2000DA000020C4110020500D002000000020B5
:108F300000D02724F40000200C0100208814002019
:108F4000E7030000EA000020F853E3A59B843E40BD
:108F500070B586B014216846FCF729F901250F4E3B
:108F6000ED03002229463046FDF7C7FC012000240E
:108F7000019002946946009503943046FDF7F8FB92
:108F80000320019002946946009503943046FDF752
:108F9000EFFB022000F086FE06B070BD000400501A
:108FA00070470000F8B5044600206A461080194D4D
:108FB00055222A70AA226A700322AA70661DEE70DA
:108FC0002A716971144A49008918AC712246E81D5A
:108FD000FCF7D4F8002007E029186A46897812883F
:108FE00089186A461180401CB042F5DB611DA81C3F
:108FF000FCF720FD01466846018029190078C871F8
:1090000068464078087221460931024800F0AAFA01
:10901000F8BD0000C8130020500D002010B51B4CF7
:10902000228A01E0891AE182E18A9142FAD2628BB6
:109030008BB253431B182383132902D14A431018C0
:109040002083208B302148436421643048431049F9
:1090500020630968401A4B2109014018E062FCF7BF
:10906000F9FA0C4A0C4BFCF76BFAFCF729FB0B499D
:10907000A062884202DD4A428018A062002801DA1C
:109080004018A06206490968486110BDD40000205C
:1090900098000020F853E3A59B843E40FF7F00002A
:1090A00088140020034A1168382389B29943014388
:1090B000116070470030014010B5FDF72BFC10BD6A
:1090C00010B59AB034216846FCF771F814210DA848
:1090D000FCF76DF81C2112A8FCF769F81B48016821
:1090E0000324E402A143C21489180160FDF770FE55
:1090F00017480169A143016106200090FF2001305B
:109100000290012003901020049002200990400456
:109110000B90000100240C900A946846FEF756F864
:109120000F200D9003200E900F94109401211194A4
:109130000DA8FDF739FF81201290032080041890BC
:10914000149412A8FDF77EFE1AB010BD0070004006
:109150004010024010480168821511430160C16847
:109160000E4A1140C16001680D4A114001608168DA
:10917000490849008160016801229204914301601D
:10918000C168FD2212049143C160002101610649BA
:109190000448886070470000001002400C40FF88BF
:1091A000F6FFF6FE0050000800ED00E070B5102458
:1091B00005252D07AC62AF20800000F07AFDAC6180
:1091C00000F0F4FF214C224EE06402E000F0EEFFDC
:1091D000E064B042FAD120780126F603002806D0D8
:1091E00001280CD0022817D003282BD128E0012217
:1091F00031462846FDF781FBFFF75AFD06E00122C4
:1092000031462846FDF779FBFFF746FB0022314641
:109210002846FDF772FB15E0A07A0122401EA072DD
:1092200031462846FDF769FBFCF7CCFD00223146AC
:109230002846FDF762FBA07A002803D1207001E0E8
:10924000FFF786F800F098FE70BD0000580000207F
:109250003001CADE10B5818CC90707D001684A68A1
:1092600001235B049A43836A1A434A60818C89070D
:1092700007D501684A6801231B049A43C36A1A434D
:109280004A60818C490707D501684A6801239B041D
:109290009A43036B1A434A60818C090707D501681A
:1092A0004A680123DB039A43436B1A434A60818C6B
:1092B000C90607D50268916801231B039943836B94
:1092C00019439160818C890607D501688A6801235A
:1092D0005B039A43C36B1A438A60818C490612D59B
:1092E00003685A6801210905046C8A4322435A60C5
:1092F000026C8A4207D10268516803235B059943D7
:10930000436C19435160818C090607D501684A688E
:109310000123DB04806C9A4302434A6010BD0000C5
:10932000F8B500260446C667FDF7EEFA0546206844
:109330000068124F000709D501212B46002249057C
:109340002046009700F054FA00280DD120680068EC
:1093500040070BD501212B460022890520460097A6
:1093600000F046FA002801D00320F8BD20206067F5
:10937000A067603426740020F8BD0000FFFFFF01E5
:10938000F8B5184CC826E078002829D16079002863
:1093900026D101206071144D686B002700281ED073
:1093A000686BC821081A15E01048E168405C6169E3
:1093B00088470F480A21008848430E490880E06822
:1093C000401CE060E068C82800DBE760696BC820EB
:1093D000401A761EE168814201D0002EE4DC6771FC
:1093E000F8BD00003C00002000000240880C002076
:1093F000E4000020F000002070B5224CE078002846
:109400003FD1207900283CD1012020711E4EF16906
:1094100000250906002933DA2156625791420AD104
:10942000F06940062CD5A079002829D0A5712089A3
:10943000401C208124E0A179002903D1A0710A20D9
:1094400000F037FC00202056CC2148430F49421839
:10945000206912181279B262401C00222061A256C3
:10946000CC235A43895881420ADC25612078401C6C
:10947000207020780E2800D12570A078401CA070A4
:10948000257170BD3C0000200038014060010020C3
:1094900010B5806A0022014640314A834A82FEF7B5
:1094A00028F910BD70B5846A606FA56F216889685E
:1094B00000260906002906DA212804D15220065385
:1094C000204600F047F820688068400606D5222D27
:1094D00004D15A200653204600F02CF8E06F1021EA
:1094E0000843E0672046FEF704F970BD10B5014659
:1094F0000968806A0968890614D400225A210A5230
:1095000001680A68FF2301339A430A6001688A6888
:10951000520852008A6001688A6840239A438A6030
:1095200020218167FEF780FA10BD10B5806AFEF732
:109530007CFA10BD01680A68FF2321339A430A6050
:1095400001688A68520852008A60202181670021E0
:109550000166704701680A68C0239A430A602021A7
:109560004167704770B5164CE278002A0CD1227919
:10957000002A09D10122E2700025C82903DC022259
:10958000A256002A01DCE57070BD0123E356CC220F
:1095900053430C4AD1500123E356CC2673439B1806
:1095A0000A460146181DFBF7E9FD6078401C607013
:1095B00060780E2800D16570A078401EA070E2E7A8
:1095C0003C00002060010020F8B504462669A2682E
:1095D000E76932436669102000253E432368324321
:1095E00078491E68784F3E4016431E6023685A68CB
:1095F00003263603B243E66832435A602368A26901
:109600008B4201D0266A32439E680B273F02BE433D
:1096100016439E606D4E23686D4AB3420CD1D268EA
:109620009207920F06D0012A38D0022A34D0032A9A
:1096300020D11EE001201DE0664EB3420AD1D2685F
:109640000C26324026D0042A28D0082A24D00C2AFE
:1096500010D10EE08B420DD1D66803229202164043
:1096600018D001229202B61A18D0B61A14D0964217
:1096700000D10820564A0126403A574FF6038B4244
:1096800036D100280CD002280DD0042812D008288A
:109690001FD11CE00020EDE70220EBE70420E9E702
:1096A000FDF738FD08E01068C00601D5384605E032
:1096B0004A4803E0FDF74EFD002873D06268510070
:1096C0005118814205D81103814202D303E030468C
:1096D000F4E7012566E0010E060250080023301869
:1096E0005941FBF71BFD03210902411A3C4A55E091
:1096F000E169B14232D1030000F07DF909070A0D9A
:1097000006250606062B0600E3E7FDF703FD1CE031
:10971000FDF710FD19E010686168C00602D5480821
:10972000304A01E0304A48088018FBF7E1FC80B27B
:1097300001462E4A10399142CBD8511C01400007F6
:10974000400F08432CE0FDF705FD616840004A0822
:10975000EAE76168012248081204E5E7030000F027
:109760004AF909070A0D06260606062C0600B0E788
:10977000FDF7D0FC1DE0FDF7DDFC1AE01068616824
:10978000C00602D54808C01902E014484A0810185B
:10979000FBF7AEFC80B20146144A1039914298D8CA
:1097A0002168C8600020206660662846F8BDFDF785
:1097B000D1FC61684A088018EAE7616848088019A6
:1097C000E6E7000000480040F369FFEF0038014081
:1097D000401002400044004000093D000024F40015
:1097E000FFFC0F0000127A000048E801EFFF0000C4
:1097F000FFB581B017460E4604460A9D09E0681C75
:1098000007D0FDF781F80499401AA8420CD8002D22
:109810000AD02068C1693046884318D00020B84279
:10982000EDD0002005B0F0BD20680168FF22A13214
:1098300091430160206881684908490081602020C7
:109840006067A0670020603420740320EAE70120ED
:10985000E5E7000010B504491020096808620248D5
:10986000FDF748FF10BD00001015002001490D2034
:10987000887070473C00002010B507480A22018A12
:1098800051438183FEF728FCFEF70AFDC8220349F5
:109890000348FEF76DF810BDD4000020880C0020AE
:1098A00010150020F8B53E4C002321783D4A1D4696
:1098B000082910D0072947D0062950D0052952D0B1
:1098C000042953D0032954D0002956D0012958D057
:1098D00002295AD05BE0A17800264A1F04E0314FEC
:1098E000BF5DFB189BB2761C9642F8DB6679277940
:1098F0009A195118E3786278C9188918C91940185B
:10990000C0430006000E1AD1012E14D0022E16D12B
:1099100025482449C018FBF731FC00F041FF6420C2
:1099200000F0C0F9BFF34F8F21492048C860BFF352
:109930004F8F00BFFDE759081046FFF733FB257036
:10994000E570A570A571F8BDA1795054491CC8B245
:10995000A071A178491F8842F5D1082001E060700C
:1099600007202070F8BDE0700620FAE7607105203E
:10997000F7E7A070E5700420F3E7552807D1012030
:10998000EFE7AA2803D10220EBE7032803D02570D4
:10999000E570A570F8BD032020702071F8BD0000AF
:1099A000CB00002064130020500D00200400FA05B5
:1099B00000ED00E010B5024A024900F0FFF810BDCA
:1099C000E1A40008200100202021020C01D0102178
:1099D0001046020A01D010460839020901D010468B
:1099E000091F820801D01046891E420801D0881E36
:1099F0007047081A704730B47446641E2578641C9A
:109A0000AB4200D21D46635D5B00E31830BC1847D3
:109A100002E008C8121F08C1002AFAD17047704737
:109A2000002001E001C1121F002AFBD1704708B5D8
:109A30000021684601706B46012202212C2000F0B3
:109A4000EFFC0221684601706B4601222C2000F0D9
:109A5000E7FC08BD38B504466D20694608706B46C2
:109A6000012207492E2000F0DBFC0649002C01D022
:109A7000054A00E0054A2E2000F0B8FC38BD000081
:109A80000608000006180000070600000716000080
:109A900038B504466B4602220021362000F08CFBCC
:109AA000B3212300FFF7A7FF0E0F08153A3A3A3A01
:109AB0001C273A3A2F34483A002168460170407812
:109AC0004108490014E06946087880088000401C7D
:109AD00004E06946087880088000801C08701DE05A
:109AE000684602780A40483202704178802001437B
:109AF0006846417012E0684602780A400270407879
:109B00004106490EF4E7694648780221084303E01C
:109B100069464878FD210840694648706B46012235
:109B20000021362000F07CFC012200AB11463620DB
:109B3000013300F075FC38BD69460878CF21084034
:109B400069462030CAE708B5032168464170012103
:109B500001706B4602220021362000F061FC0122D8
:109B6000D20306212D2000F041FC012000F09AF8DC
:109B70000120FFF78DFF08BD08B5020A69464A704B
:109B800008706B46022204212D2000F049FC0320BE
:109B9000694608706B46012206212D2000F040FC2A
:109BA0000020694608706B46012206212D2000F036
:109BB00037FC0A212D2000F0E5FA08BDF8B516465D
:109BC0000F460446002503E03946B047641C6D1C6F
:109BD00020780028F8D12846F8BD0000F8B54A00E2
:109BE0002B4B520DD6182B4A0C460546142E2BDA59
:109BF000002E12DA284BFBF789FB00221346FBF7F5
:109C0000AFFE40D2002C03DA0124E40700253AE03D
:109C10002046284337D0214C14E0214F0B46F74013
:109C20003B402B4331D01C4BFBF770FB002213460B
:109C3000FBF796FE27D2002C03DD01200005F04043
:109C40000419BC4300251EE0332E1EDC33460027DA
:109C5000143BFF43DF40384217D00F4BFBF700FCAB
:109C600000221346FBF77CFE0DD2002C0ADD142ED9
:109C70000CD03420811B012088404019A84200D21A
:109C8000641C0546BD4321462846F8BD641CF9E71F
:109C900001FCFFFF9C7500883CE4377E0000F03F2C
:109CA000FFFF0F007D2110B5C900484300F001F807
:109CB00010BD002140E000BF00BF00BF00BF00BFDB
:109CC00000BF00BF00BF00BF00BF00BF00BF00BF9C
:109CD00000BF00BF00BF00BF00BF00BF00BF00BF8C
:109CE00000BF00BF00BF00BF00BF00BF00BF00BF7C
:109CF00000BF00BF00BF00BF00BF00BF00BF00BF6C
:109D000000BF00BF00BF00BF00BF00BF00BF00BF5B
:109D100000BF00BF00BF00BF00BF00BF00BF00BF4B
:109D200000BF00BF00BF00BF00BF00BF00BF00BF3B
:109D300000BF00BF00BF491C8142BCD37047000078
:109D4000FEB5044600200190009060797349400000
:109D50000E5A61782578491E7148CFB20163042DEF
:109D600077D0072D75D000210291217801736C49BD
:109D7000E379012292058969002B6CD091438161BE
:109D80006748217A4173217A82698907890B0A43DE
:109D900082610021042000F034FB324661492E200C
:109DA00000F024FB3846FFF755FE5F4E0522705D3C
:109DB000810040185D49431807212B2000F030FB3B
:109DC0005B49029801220B180B21282000F028FB88
:109DD000705D584980000A580C21282000F011FBC2
:109DE000E079554980004018A1794900425A022182
:109DF000272000F0FBFA51487E00825B04212720D7
:109E000000F0F4FAE079002829D0A07804282CD0BA
:109E100028206946087220220621272000F0E6FA51
:109E200002AB01222621272000F0FAFA444938012A
:109E30004018E178890042580821272000F0E1FA13
:109E4000A17A601C627A0902114313D016E000E087
:109E500001E0012188E71143F608816190E764225F
:109E60000621272000F0C2FAE0E7102069460872B8
:109E70000246D1E733490172090A4172417A007AF8
:109E80000A0202432021272000F0B0FA2E4F0C21B5
:109E900023203A6800F0B5FAF019828804212320C3
:109EA00000F0A4FAA07900280BD0E079274901221C
:109EB00043180021212000F0B3FA03200190012073
:109EC00000902A07120F10010243607800218007DA
:109ED000000B02430198000502430098400402432E
:109EE0002079C006400902436079C00602431F2062
:109EF00000F087FAA078617801230843020408483B
:109F0000DB030261E179490319430A43026100213D
:109F1000082000F076FA0020FEBD00006CA80008C2
:109F2000240100200428000014A800080C000020D0
:109F30002A0000201CA800083CA8000848A8000827
:109F40004CA800084110000034A800082C00002094
:109F500038B50C4607498A8B002102432C2000F0BB
:109F600045FA684604706B46012206212C2000F059
:109F700057FA38BD2401002010B5FFF758FD10BD79
:109F800010B504460421362000F0FCF80121C90276
:109F9000002C01D0084300E088430246042136200B
:109FA00000F02FFA10BD000038B540206946087057
:109FB00000210E2000F0E6F80446002211460E2093
:109FC00000F01FFA6B46012200210D2000F028FA54
:109FD000074A00210F2000F014FA00F0EDF92246A4
:109FE00000210E2000F00DFA02480021017338BD57
:109FF000F8FF272444010020FEB5054604206946E9
:10A000000870514C00206075214620312063487152
:10A010000873A0836063A06300F0C8F84B4E206013
:10A0200002E000F0C3F82060B042FAD10020FFF750
:10A030002FFD00F0BBF8464E20603078242801D96F
:10A04000243806E00621FBF753F80622101A4001D7
:10A050000843020601040A4301020A430243B260B4
:10A06000706000211E2000F0CCF900F09FF8206005
:10A070006B4601220021242000F0D2F91E20FFF7B8
:10A080007BFD86B2300AA0730420FFF775FD0746FA
:10A0900000F08CF820603806000E0DD002206946D2
:10A0A000087101AB012212212D2000F0B9F9A08B1B
:10A0B000012109030843A08300F078F820600620FE
:10A0C000FFF75AFD60600720FFF756FDA060F0061D
:10A0D000C00E207501D110202075C0B200F0DCF94F
:10A0E000E80707D0FFF72FFDA08B0121C902084325
:10A0F000A0830AE00521362000F02EF8154908401B
:10A1000002460521362000F071F90120FFF7C0FC5E
:10A110000021042000F036F8A0610021262000F084
:10A1200031F815218903084302460021262000F05A
:10A1300068F900222621362000F058F900F036F8A0
:10A1400020600020FEBD0000240100203001CADE96
:10A1500000000020FFFD000038B5094C89B280B234
:10A160006B46022200F028F8002806D168464078A5
:10A17000010268460078081884B2204638BD000005
:10A18000FFFF000038B50024E44389B280B26B467B
:10A19000042200F011F8002806D103216846435C30
:10A1A0002202D418491EFAD5204638BD10B5002128
:10A1B0000846FFF7E7FF10BD38B5002909D0402455
:10A1C00020436C462070C8B27F2906D860700220F8
:10A1D0000AE069460870012006E0802420436C46AE
:10A1E0006070C809A0700320694600F0B3FA38BD5A
:10A1F00010B5144603460A4621461120FFF7DCFF3E
:10A2000010BD10B50346052200211520FFF7D4FF2D
:10A2100010BD10B50346052200211720FFF7CCFF23
:10A2200010BD38B5054600206946087000F0C4F836
:10A23000FF2401342246002D01D003221202002106
:10A240000D2000F0D3F8002D13D06B46012203211E
:10A250000F20FFF7B1FF68460078000709D5FFF728
:10A26000A3FE224600210D2000F0C0F80020C043CC
:10A2700038BD002038BD10B5024601210A2000F08B
:10A28000C0F810BD10B5044600211A20FFF77AFF70
:10A29000000D22030005120B024300211A2000F0DA
:10A2A000B0F810BD10B5024602492E2000F09EF80D
:10A2B00010BD000004180000F8B505466B460122E9
:10A2C00003210420FFF778FF0126114C3607002DEB
:10A2D0000DD02A4600210C2000F088F86946087845
:10A2E0001021084369460870A069304307E06946B9
:10A2F0000878EF21084069460870A069B0430B4612
:10A30000A06101220321042000F08AF8F8BD0000BA
:10A310002401002010B502460021182000F066F844
:10A3200010BD0000F8B50746002568460570B8075F
:10A33000204C2E4600280ADA8020694608706B46B9
:10A34000012200210D2000F06BF801202073F80796
:10A350006946087821D006210843694608706B4693
:10A36000012200210D2000F05BF803210F20FFF7F0
:10A37000F3FE8121C900084219D0402069460870C7
:10A380006B46012200210D2000F04AF80020FFF763
:10A39000F7FD00252673ED4309E0022108436946D5
:10A3A00008706B46012200210D2000F039F8284684
:10A3B000F8BD0000440100201CB56B4601220321BA
:10A3C0000F20FFF7F9FE684600784022C1091040CF
:10A3D000C9014000814208D0012069460871024647
:10A3E00001AB03210D2000F01BF81CBD08B56B4626
:10A3F0001A70120A5A7089B280B2022200F010F864
:10A4000008BD38B500236C46E254120A5B1C042BCD
:10A41000FADB89B280B22346042200F001F838BD8D
:10A4200038B58024002909D0C02528436D462870FE
:10A43000C8B27F2907D86870022009E02043694626
:10A440000870012004E020436870C809A870032048
:10A45000694600F0BBF938BD10B514460123121847
:10A460009B029A4202D90020C04310BD0B46821EB7
:10A4700021460920FFF7D4FF002010BD10B5054A82
:10A480008905126901430A4300210820FFF7B9FF3B
:10A49000002010BD2401002038B504466B4601227F
:10A4A0000E212B20FFF788FE68460078E106400960
:10A4B0004001C90E0143684601706B4601220E211E
:10A4C0002B20FFF7ADFF38BD10B5002142541C060C
:10A4D000120A22431B0A491C0429F7DB10BD0000A5
:10A4E00013B501231A4669460248FDF79FFA009802
:10A4F0001CBD0000101500207CB5002425466846D0
:10A50000FFF77FFE04206946220E2D02154322022A
:10A510000C5C1443401EF7D5204629467CBD7CB513
:10A52000002425466846FFF774FE04206946220E83
:10A530002D02154322020C5C1443401EF7D5204621
:10A5400029467CBDFCF7EEF9FEF7BAFDFDF7D8FD14
:10A550003F494048002522C005608561C5613E49EC
:10A560000562C1600838FCF761FBFDF7B5FDFDF73A
:10A5700097FEFDF773FEFDF77BFD052601223607EA
:10A58000D1033046FCF7B9F9FEF716FBFDF774FC72
:10A59000FBF7B0FAFBF77EFA0721B015FFF7D8FCFE
:10A5A0002E4C0A21208A01224843A0831103304601
:10A5B000FCF7A3F92748C82229498830FDF7D8F9C4
:10A5C000284F294E207900283FD0607800283CD0C1
:10A5D000FEF776FD2571FBF77DFC20700F280AD968
:10A5E000012211033046FCF788F9FEF7DFFD002257
:10A5F0000121090309E0012251033046FCF77DF9EE
:10A60000FEF7D4FD0022012149033046FCF775F91D
:10A61000FDF776FBA08B002801D0401EA0831348D5
:10A62000A18B00780843CDD13878002801D00328C9
:10A63000C8D10121C9023046FCF756F90028C1D122
:10A6400001210846FCF7E4FBBCE7FDF759FBB9E73D
:10A65000007C004088140020FFFF0000D400002090
:10A66000880C00206A0000200004005042000020F6
:10A6700010B586B01748FCF75EFA14216846FAF761
:10A6800096FD1548009003200190002002900520BF
:10A6900069460007FCF76CF869461048FCF768F853
:10A6A00069460F48FCF764F801210846FCF7B0FB47
:10A6B000FF2401342046FCF783FB0A490868042282
:10A6C000104308602046FCF78BFBFCF791FB06B0BB
:10A6D00010BD000088140020FFFF0000000400509F
:10A6E000000800500070004010B501229202164987
:10A6F0001648FBF78DFA1448154902888A4221D082
:10A700000180FF2101318180FF21F531C1800A21C3
:10A71000018100211E224181D24382810122C28116
:10A7200081831E23C386022303877823438782877E
:10A73000C28702464032118451849184C183918042
:10A7400000F02EF810BD0000500D002000FC0008A5
:10A75000AA550000F0B58C460025102605210907F2
:10A760008E620E4C08E067467F5DE760A768FF07D2
:10A77000FCD0E7681F706D1C8542F4DB00200746A3
:10A7800006E0E760A568ED07FCD0E5681D54401CB5
:10A790009042F6D38E610020F0BD000000300140F1
:10A7A00070B572B60124074DA40221462846FBF776
:10A7B00015FA002804D0224603492846FBF7B2FACE
:10A7C00062B670BD00FC0008500D0020F0B50025F9
:10A7D000102605279C463F070B46BE620C4C06E040
:10A7E000595DE160A168C907FCD0E1686D1C854234
:10A7F000F6DB002007E06146095CE160A168C9075B
:10A80000FCD0E168401C9042F5D3BE610020F0BD51
:10A81000003001400000010203040005405C00001C
:10A82000A05C0400C06C0800805C0400E03F1E00D7
:10A83000E07D1E0007A9022570889B880A0016008B
:10A84000010006000100020087008D002D001A3172
:10A8500052001A339A001A351D011A376B003B312A
:10A86000BE003B335E013B3596023B3700009959F1
:10A870009959EB518F421E45142E0080EB51F5285B
:10A880003333E13A703DE13AC235852BC23533337B
:10A89000C235C235AE47E13A5138A33051380000D5
:10A8A0000000000000000102030406070809030479
:10A8B00006080C10182030000000000102030400FC
:10A8C000E0A800080000002024010000109A000801
:10A8D00004AA00082401002014190000209A00088E
:10A8E0000000000000000000000000000704000954
:10A8F0001E0805400826091040085608054008268D
:10A900001D040008BE1D040008BED8BC401008008D
:10A91000010000000000C84200000000000000002C
:10A920000000000000000000000000000000000027
:10A930000000000000000000000000000000000017
:10A9400000000000000000000000000000005C1299
:10A9500000000000000000000000000000000000F7
:10A9600000000000000000000000000000000000E7
:10A9700000000000000000000000000000000000D7
:10A9800000000000000000000000000000000000C7
:10A9900000000000000000000000000000000000B7
:10A9A0000202040009090102008100000000000009
:10A9B0000100000000000000000000000000000096
:10A9C0000000000000000000000000000000000087
:10A9D0000000000000000000000000000000000077
:10A9E0000000000000000000000000000000000067
:10A9F0000000000000000000000000000000200037
:04AA00000000000052
:04000005080050C1DE
:00000001FF
